:10015F007B027D407F011201007D407F011201B8BB
:10016F007F011202297F0312028AE4FFFEE4FDFCE5
:10017F000DBD00010CED64644C70F50FBF00010E56
:0F018F00EF64644E70E77D407F011201F780DB63
:1001E300E4F59AF591F5A1F59BF592F5A2F5A0F545
:0401F30090F58022E1
:10010000EF701CEB7006EDF4529A529BBB0107EDA9
:10011000F4529AED429BEB64027043ED429A22EF57
:100120006401701CEB7006EDF452915292BB010712
:10013000EDF45291ED4292EB64027022ED42912275
:10014000EF64027019EB7006EDF452A152A2BB01EC
:0F01500007EDF452A1ED42A2BB0203ED42A12242
:10020A00EF70028D80BF01028D90BF02028DA02285
:1001F700EF7003ED4280BF0103ED4290BF0203EDB4
:0302070042A022F0
:1001B800EF7004EDF45280BF0104EDF45290BF02D9
:0601C80004EDF452A02238
:0F021A00EF7003AF8022BF0103AF9022AFA0228D
:1001CE00EF7005E5805DFF22BF0105E5905DFF2222
:0501DE00E5A05DFF2219
:04029200E4F5CF229E
:08028A00E5CF54F84FF5CF2237
:0402960043CF102220
:0E02290075FEC1EF700453FF7F2243FF802259
:0E02370075FEC1EF700453FFBF2243FF40224B
:0B02530075FEC2E5FF54BF4FF5FF220F
:0B025E0075FEC1E5FF54CF4FF5FF22F5
:0E02450075FEC1EF700443FF082253FFF7223D
:0B02690075FEC1E5FF54F84FF5FF22C1
:0B02740075FEC2E5FF547F4FF5FF222E
:0B027F0075FEC2E5FF54F34FF5FF22AF
:0300000002019E5C
:10019E0078FFE4F6D8FD9000007F007E01E4F0A326
:0A01AE00DFFCDEFA75810702015F35
:00000001FF
